:1000000004EF00F0FFFFFFFF0AEC02F0430E656E05
:100010006F0E666E6E0E676E740E686E720E696E8F
:100020006F0E6A6E6C0E6B6E650E6C6E200E6D6ED2
:10003000640E6E6E650E6F6E200E706E740E716EB5
:10004000650E726E6E0E736E730E746E690E756E43
:100050006F0E766E6E0E776E200E786E640E796E71
:10006000650E7A6E200E7B6E620E7C6E610E7D6E6A
:10007000740E7E6E740E7F6E650E0001806F720EC0
:10008000816F690E826F650E836F0A0E846F0D0E8D
:10009000856F866B490E876F4E0E886F490E896F8C
:1000A000540E8A6F200E8B6F750E8C6F730E8D6FD2
:1000B000610E8E6F720E8F6F740E906F200E916FA7
:1000C000350E926F360E936F300E946F300E956F23
:1000D000300E966F620E976F640E986F730E996F65
:1000E0000A0E9A6F0D0E9B6F9C6B4D0E9D6F650EE9
:1000F0009E6F730E9F6F750EA06F720EA16F650ECF
:10010000A26F200EA36F410EA46F440EA56F430E85
:10011000A66F300EA76F3D0EA86F200EA96FAA6BB9
:100120004D0EAB6F650EAC6F730EAD6F750EAE6F8F
:10013000720EAF6F650EB06F200EB16F420EB26FD0
:10014000610EB36F740EB46F740EB56F650EB66F3B
:10015000720EB76F690EB86F650EB96F200EBA6F69
:100160003D0EBB6F200EBC6FBD6BD1EC03F00A0ED1
:10017000AF6EAC84EAEC03F079EC03F015C0BEF08E
:1001800016C0BFF0650E0001C06F000EC16F53ECCA
:1001900003F000C015F001C016F079EC03F015C0B3
:1001A000BEF016C0BFF0870E0001C06F000EC16F19
:1001B00053EC03F000C015F001C016F079EC03F029
:1001C000040E0C6EFF0E0B6EFF0E0A6E0C2E01D08D
:1001D00007D00B2E01D003D00A2EFED7FAD7F6D7C0
:1001E000300E0B6EFF0E0A6E0B2E01D003D00A2EBE
:1001F000FED7FAD7880E0A6E0A2EFED7000000003E
:10020000616A612A61C0BEF0000E0001BF6F15C0B7
:10021000C0F016C0C1F0A1EC02F079EC03F0090EB9
:100220000001C46FDFEC03F00001BE6B2BEC03F0A8
:1002300000C062F001C063F015C0BEF016C0BFF090
:100240009D0E0001C06F000EC16F53EC03F000C0A3
:1002500015F001C016F079EC03F062C0BEF063C087
:10026000BFF015C0C0F016C0C1F0A1EC02F079ECEF
:1002700003F0090E0001C46FDFEC03F08290040E5E
:100280000C6EFF0E0B6EFF0E0A6E0C2E01D007D007
:100290000B2E01D003D00A2EFED7FAD7F6D7300E98
:1002A0000B6EFF0E0A6E0B2E01D003D00A2EFED766
:1002B000FAD7880E0A6E0A2EFED700000000828050
:1002C000A80E046E000E056E62C000F063C001F05F
:1002D00099EC03F000C064F024D00001FF0E816EA1
:1002E00039D00001FE0E816E35D00001FD0E816E09
:1002F00031D00001FB0E816E2DD00001F70E816E12
:1003000029D00001EF0E816E25D00001DF0E816E35
:1003100021D00001BF0E816E1DD00001FF0E816E45
:1003200019D06450000AD9E06450010ADAE0645040
:10033000020ADBE06450030ADCE06450040ADDE0FA
:100340006450050ADEE06450060ADFE06450070AE4
:10035000E0E0E3D7000162C000F063C001F02B0EC3
:10036000046E000E056E02EC03F00A0E046E0450DB
:10037000000105E001320032019EFF0FF9D7650E42
:100380000024626E000E0120636E15C0BEF016C020
:10039000BFF0AB0E0001C06F000EC16F53EC03F055
:1003A00000C015F001C016F079EC03F062C0BEF099
:1003B00063C0BFF015C0C0F016C0C1F0A1EC02F0E0
:1003C00079EC03F00D0E0001C46FDFEC03F00D0EAD
:1003D0000C6EFF0E0B6EFF0E0A6E0C2E01D007D0B6
:1003E0000B2E01D003D00A2EFED7FAD7F6D7BF0EB8
:1003F0000B6EFF0E0A6E0B2E01D003D00A2EFED715
:10040000FAD72B0E0A6E0A2EFED70000000000005D
:10041000F8D6FFD70A0E176E4D0E186E690E196EBC
:100420006B0E1A6E720E1B6E6F0E1C6E430E1D6EDF
:10043000200E1E6E310E1F6E380E206E460E216E7F
:10044000320E226E350E236E320E246E200E256E75
:10045000510E266E3D0E276E310E286E300E296E1F
:100460004D0E2A6E680E2B6E7A0E2C6E200E2D6E9F
:10047000610E2E6E760E2F6E650E306E630E316E2F
:10048000200E326E620E336E6F0E346E6F0E356E4E
:10049000740E366E6C0E376E6F0E386E610E396EDE
:1004A000640E3A6E650E3B6E720E3C6E3A0E3D6EF9
:1004B000200E3E6E3F6A170E156E000E166E2E0E43
:1004C000406E2E0E416E2E0E426E2E0E436E2E0E7E
:1004D000446E2E0E456E2E0E466E2E0E476E2E0E5E
:1004E000486E2E0E496E2E0E4A6E2E0E4B6E2E0E3E
:1004F0004C6E2E0E4D6E2E0E4E6E2E0E4F6E2E0E1E
:10050000506E2E0E516E2E0E526E2E0E536E2E0EFD
:10051000546E2E0E556E2E0E566E2E0E576E2E0EDD
:10052000586E2E0E596E2E0E5A6E2E0E5B6E2E0EBD
:100530005C6E2E0E5D6E5E6A400E5F6E000E606E2B
:100540001200C0C0E1FFC1C0E2FF200EE66E010E46
:100550000001C025E16E000EC121E26E200EE66EA4
:10056000020EC025E16E000EC121E26E200EE66E85
:10057000030EC025E16E000EC121E26E200EE66E74
:10058000040EC025E16E000EC121E26E300EE66E53
:10059000050EC025E16E000EC121E26EE66A040E72
:1005A000C26F000E006EBF51005C02E1BE51000838
:1005B00028E2C251C025E16E000EC121E26E0A0E92
:1005C000046E000E056EBEC000F0BFC001F099ECD5
:1005D00003F008C000F009C001F0300E002600C092
:1005E000E6FF0A0E046E000E056EBEC000F0BFC02E
:1005F00001F099EC03F000C0BEF001C0BFF0C207EB
:10060000D0D7120000010B6A0A6A096A005004027E
:10061000F4CF09F0F3CF08F001500502F4CF0BF04E
:10062000F3CF0AF000500502F3500926F4500A22D5
:10063000E86A0B2201500402F3500926F4500A2202
:10064000E86A0B2208C000F009C001F00AC002F0FD
:100650000BC003F01200C26AC00EC212C18CC18E60
:10066000BEC000F0003600900036009000360090CA
:100670000050C212C280F5EC03F0C284C2B4FED7AF
:10068000080E026EC4CF00F0000E016E025005E0AD
:10069000003600900136FF0FFAD7C3500012000E4B
:1006A0000112C2901200BEC0C2F0BFC0C3F0C2C0EF
:1006B00002F0C3C003F00001C24BC32BC0C0E9FF6E
:1006C000C1C0EAFFC04BC12BEECF00F002C0E1FF7A
:1006D00003C0E2FF00C0E6FF02C0E9FF03C0EAFF7B
:1006E000EECF00F00052E3E1BEC000F0BFC001F069
:1006F000120015C0C4F016C0C5F0B7EC03F000C07E
:10070000BFF00001BE6BBE511524E96E000EBEBFE6
:10071000FF0E1620EA6EEECFC4F0DFEC03F000010E
:10072000BE2B800EBE19006E800EBF19005CEBE37D
:1007300012000001086A096A100E0C6E01340836B6
:1007400009360450085E0550D8A0053C095ED8B0B3
:10075000B1EF03F0045008260550D8B0053C092637
:10076000D890003601360C2E9EEF03F01200C4C064
:10077000C6F0C5C0C7F0C6C0E9FFC7C0EAFF0001A8
:10078000C64BC72BEECF00F00052F5E1C451C65D59
:10079000006EC551C759016E010E005E000E015A70
:1007A0001200816A936AFF0E806EFF0E926E010E38
:1007B000C26E880EC16E826A8B6A946A1200016AE8
:1007C000ACB2012A0150000A02E10000F8D7C4C00F
:1007D000ADFF1200AC8A900EAB6E948E949C9EAAD4
:1007E00003D0AECFC2F0FBD71200120E0A6E0A2E53
:1007F000FED71200FFFFFFFFFFFFFFFFFFFFFFFF1E
:020000040030CA
:0E000000FFF9FEFEFFFFFBFFFFFFFFFFFFFF0C
:00000001FF
